:040000006F20D0009D
:100004000000000000000000CA090000CC09000044
:10001400000000000A2800000000000000000000AA
:100024000A2800000A280000000000000000000068
:100034009E0B0000000000000A28000000000000E1
:100044000A2800000A2800000A2800000A280000E4
:100054000A2800000A2800000A2800000A280000D4
:100064000A2800000A2800000A2800000A280000C4
:100074000A2800000A2800000A2800000A280000B4
:100084000A2800000A2800000A2800000A280000A4
:10009400961D00000A2800000A2800000A28000013
:1000A4000A2800000A2800000A2800000A28000084
:1000B4000A2800000A280000260200000A2800007E
:1000C4000A2800000A2800000A2800000A28000064
:1000D4000A2800000A2800000A2800000A28000054
:1000E4000A2800000A2800008A1D00000A280000CF
:0C00F4000A2800000A2800000A2800006A
:10010000397101436EC619A0397141536AC866CA74
:1001100062CC5ECE19A0397101535AD056D252D456
:100120004ED64AD826DA22DC06DE330161408282CE
:1001300041114AC026C222C406C68282B24D410184
:10014000024D924C224CB24B4101024B924A224A40
:10015000B2494101024992442244B24041018280A5
:100160003D432A876373C3029377F700BDEFADE584
:10017000937606FF3D8ABA960CC34CC30CC74CC796
:100180004107E36BD7FE11E28280B306C3408A06C3
:100190009702000096966780A6002307B700A30683
:1001A000B7002306B700A305B7002305B700A304D3
:1001B000B7002304B700A303B7002303B700A302CB
:1001C000B7002302B700A301B7002301B700A300C3
:1001D000B7002300B700828093F5F50F9396850052
:1001E000D58D93960501D58D61B79396270097021B
:1001F000000096968682E78086FA9680C1171D8F4A
:100200003E96E374C3F8A5B79387418A03C7F70303
:1002100003C7E70303C7D70303C7C70303C707041D
:1002200083C717048280B717004079572398E78067
:100230009387078073002030EFF29FEF01111306C0
:10024000000281450A85293F1165EF20F0213724FE
:10025000014013050440EF208063B7070E003EC63F
:100260008A85854713050440230AF10002C002C2B3
:1002700002C402C8EF20A0659D4605461305044050
:10028000A145EF20A06C854513050440EF2080694F
:100290000561C9B5EFF2DFE9372501408545130552
:1002A0000540EF2020697DB5EFF29FE80564B72493
:1002B00001407D141389044089454A85EF2000756B
:1002C00019E511E041BD7D1442044180F5B77DD8A8
:1002D00013850440EF2000732391A184E5B7EFF26A
:1002E0009FE313890184834709009306F00F638E0F
:1002F000D7000544638D870691CB138A0184094793
:100300006384E7080D476384E71081B5B7140140A3
:1003100013850480930700025CC923AA84C0370AAE
:1003200000202300890023A884C093090A00239099
:10033000F90093050A009307800223A4F90093842F
:1003400004C0EF20607293050A002685239089007F
:1003500023A40900EF204071353FB707002003C7F1
:10036000070C2382E18485472300F90079BF83C706
:1003700041841384418489E7313F89472300F90090
:100380001C20FD171CA051B70537B70400201389A6
:100390000400C147B71901402324F90093850400E4
:1003A00093070002138509802310F900EF20C06B2A
:1003B00093850400138509C023108900EF20C06ACB
:1003C00083D621840567B707002013060799938712
:1003D000070C6376D60298239306F003050713777C
:1003E000F70F63E4E60098A311A094A39C2393C79E
:1003F000F7FF2382F1848D472300FA0039B71307F2
:10040000F788E365D7FE982375D37D17E9BF03C747
:1004100041849387418419E3230009007D1798A341
:10042000EDB5B707002003C5070C82801387C1CE46
:10043000A94614A3AD4654ABB1462304D702B54632
:10044000230ED702B9462308D7041306470693861E
:10045000C1CE91453715014005481C230CB38328B4
:1004600085C0BD8BB317F800B3F7170189E79C323D
:1004700093E787009CB25107E311C7FE8280EFF239
:100480009FC941691384C1CE8144371A0140854A0E
:10049000114B7D199549182003268AC01C303D8BCD
:1004A0003397EA00718F93F687002DEF3A206304AB
:1004B000270105073AA03A2063FCE90413F6170068
:1004C00011EE93E716001CB01C44B9C3B1E22685B7
:1004D00082971C3093E707011CB01DA85220636966
:1004E000C70213F7270019C37A201DC393E727001B
:1004F0001CB05C4481CB99E6268582971C3093E73B
:1005000007021CB07A203E2063FBE70023110400A1
:10051000850493F4F40F5104E39F34F73DB1998FB0
:100520003EA0FDB7918BEDF71C48A3006401231199
:100530000400F9DFF1FE268582971C3093E707045B
:1005400061BFEFF2FFBE938701D50947D8C33715C6
:1005500001401307800298C7938501D513070060F7
:10056000130505809AA3EF202050EDB6EFF25FBC93
:1005700083D561843145EF20004BEF20B009D9BE0F
:1005800083C7518485E3EFF2BFBAB7170140214713
:1005900023A8E780938761849A23136717009AA39F
:1005A000F1374DBE8280EFF2BFB8B7170140214747
:1005B00023AAE780938761849A23799B9AA37D3746
:1005C00051BEB717014003A5C7800D810589828000
:1005D000EFF21FB6FD3719C1F937ADBE5537F5BF7C
:1005E000EFF21FB5B7170140414723A8E7C0938733
:1005F00061849A23136727009AA38D3FA1BEEFF26F
:100600003FB3B7170140414723AAE7C093876184EE
:100610009A23759B9AA3993F35BEB717014003A54E
:10062000C7C0118105898280EFF29FB0FD3719C1E3
:10063000F9370DB67537F5BFEFF29FAF3145EF20B3
:100640004040938461848AA0EF20C07C9A20ED779B
:10065000938707F0F98F2D67130707F013846184E0
:100660006387E700ED77938737F01EA001371E20E0
:10067000858B91C331371E20898B91C39537D9BCA7
:1006800041111387818481471385C1849386018535
:100690000543130EF00F8D483306F50010220C238E
:1006A000328881C5FD1513F8F50F2300070101CE2F
:1006B000630BC609631DC800B385F600902113467D
:1006C000160090A129A03386F60023006600850756
:1006D0000507E39317FDB7072000938787023EC401
:1006E000930740027C869387C1CE03C7970283C6D7
:1006F000D7039305E100058B858A3C0001C792234F
:10070000098292A399C2239007008907E398B7FE54
:1007100013870185342393870185014791C2388669
:10072000B7060040DABA9433014791C23885B7065C
:1007300000409ABE9823814711C33C84370700408C
:100740005EBF410182803386F6002300060041B778
:10075000EFF21F9EBD35133515001384C184330598
:10076000A04008B05D3D133515003305A04008A03A
:10077000013FCDB2EFF2DF9B011102C49307F03FBE
:100780004C00370500407C8402C22316010002C8D9
:1007900002CA02CC02CEEF20206BC1679387070606
:1007A0003EC88145894737050040FC84231B010072
:1007B000EF20F00D814537050040EF20300E8145D8
:1007C00037050040EF20F00E854537050040EF204B
:1007D000700A0C0837050040EF20A06D0C083705A3
:1007E0000040EF20A0730C0837050040EF20607C2C
:1007F000854537050040EF209006B707004023925B
:100800000702854537050040EF20F0039387C18438
:100810007D579AA3B8A305616FF0DF9393773500F6
:1008200099EF130740063377E502854719E79307E9
:1008300000193375F502933715003E858280814794
:10084000EDBFEFF27F8C835A0500130710089387E2
:10085000EA84C207C1836361F70CB739E101378AC3
:10086000E2012A8981441304207B93890938130A01
:100870000A50639B8A06834929000D6BD56AFD19CE
:10088000014A93F9F90F130B4B17938A0A18054C79
:10089000931B0A0193DB0B0163E23B07034449000E
:1008A0008567938707E13304F402834759001307F0
:1008B000C0030545B387E7025567130707183E9441
:1008C000834769003E9483473900FD17B387E702E9
:1008D0003E942694EF20E0372285EF20404EEF2013
:1008E000605301456FF0DF8522850D3F11C5D2941D
:1008F000050442044180B5BFCE94DDBFB3074B0170
:100900009C232285B3875703BE94093F01C5639397
:100910008B01D694050AADBF7D55E9B7EFF25F8133
:100920000545EF2000332145EF20A011A389A184C4
:10093000EF20404E1145EF20C01085679387773335
:10094000630DF506EF20200D0545EF200033B707B6
:10095000002003A4470C938431857D59058013053D
:100960001004EF20404031ED7D14E31A24FF1305FD
:100970000010EF2000330545EF206033EF20804961
:10098000EF20404AEF20004121657D15EF20A04572
:10099000EF204048138501836D35EF20C040854727
:1009A000854521459CA0EF200008EF20A0468565E5
:1009B000938575331145EF200007EF20A0450145D1
:1009C00019A07D554DF46FF0EFF801A001A083C789
:1009D000D1D3858B91E7EFF2AFF5DD3E6FF08FF766
:1009E000828083C7D1D3858B91E7EFF26FF42D39E5
:1009F0006FF04FF68280EFF20FF241110545EF20C4
:100A0000E024752C3705201885450505EF20E02FDB
:100A100085451305D022EF20602D056B8545130514
:100A20000B80EF20C02A89473EC4930780023EC650
:100A30004C00896737150140371401407C8223132D
:100A40000100EF206002130504408D474C007C82BA
:100A5000EF208001130504809307001C4C00E17A0D
:100A60007C82EF206000130504C093876A024C006B
:100A70007C82EF10707F930404809D476147232898
:100A8000F4804C0026853AC67C82214AEF10D07D46
:100A90004149232A44814C0026854AC6231241013C
:100AA000EF10907C93070002232AF48085494C00C4
:100AB0002685130404C07C82EF10107B232A3401A6
:100AC0004C00228523123101EF10107A4C00232AAA
:100AD0002401228523122101EF101079930780044D
:100AE0004C0026853EC623122101EF10F07793C7F4
:100AF0000AC04C0022857C82EF10107791474C0091
:100B000026853EC623125101EF1010764C00228537
:100B100023124101EF10507585450945EF20E00390
:100B20004C009307003022853EC64EC4EF10D073B0
:100B3000F533EFF0BF8F371700009387C1CE13074F
:100B4000E79C98C7371700001307279ED8CFEFF010
:100B50005F9FDD340531EFF02FEEB707002083A74C
:100B6000470C81460147A1831386F7FFB7F700E0E2
:100B700090CBD4CB814694C7D8C73D4798C323A216
:100B80000700B7E700E023A0671137F700E08327ED
:100B900007D1DD9B2328F7D073005010CDBF411142
:100BA00022C6938641859C2213844185850793F74D
:100BB000F70F9CA295EF938781859843050798C30B
:100BC00083C7D1D3858B8DC7EFF0BF859307000313
:100BD00063F6A700EFF03F9DEFF07FA2EFF07F8478
:100BE0009307000263E6A700EFF09F99EFF05F9F85
:100BF000EFF0EFEEEFF0BF881C208D8B91E3893E84
:100C0000B7F700E023A20700DC4391C301A0324400
:100C1000410173002030B71702409843B706FFF038
:100C20001367170098C3D843758FD8C39843B70686
:100C3000F7FEFD16758F98C39843B706FCFFFD16A7
:100C4000758F98C3D843B70601FFFD16758FD8C3BB
:100C500037079F0098C7B746024003A7068013676F
:100C6000070123A0E680D843B706C1FFFD16D8C30D
:100C7000D843D8C3D84313670740D8C3D843758F28
:100C8000D8C3D843B7061000558FD8C39843B706CA
:100C90000001558F98C3984393166700E3DD06FE65
:100CA000D843B7160240719BD8C3D84313672700B7
:100CB000D8C32147DC42B18BE39EE7FE8280B716A2
:100CC0000240DC421146B18B138741806385C70027
:100CD00021466388C702B7177A00938707201CC391
:100CE000B7170240DC43918393F6F700B707002063
:100CF0009387C700B69794231C43B3D7D7001CC370
:100D00008280DC42D4424166C983BD8BF18E890763
:100D100045466393C700C94781EEB746024083A6A4
:100D20000680C18A89CEB7167A009386062021A84C
:100D3000B7160240D4421396E600E35606FEB716F5
:100D40003D0093860690B387D70251BFEFF24FBEA6
:100D500019E583A7418605479AAB6FF0AFBF83A71C
:100D6000C1869C43829703A541862905FDB7EFF212
:100D70002FBC19E583A7418605479AAB6FF08FBD5D
:100D800083A7C1869C47829703A541863105FDB79D
:100D900003A7418601E589471EAB8280EFF24FB978
:100DA000239001861C231384018693F7F7079DE7A0
:100DB00018379377070299C389471CA01377070454
:100DC0001C2019CB93E717001CA083A7C1869C4B5E
:100DD000829722856FF00FB8F99BFDB78546138582
:100DE0000186E389D7FE89460145E395D7FE58334E
:100DF000B7660040938606C09377F7008A07B697D8
:100E000062079C4361876359070093F707034147D3
:100E1000E39DE7FA85474DBF0D67F98F0567CDBFA5
:100E2000EFF26FAF83A441863E8A822831E898248E
:100E300091476317F7041387C18514438547639C63
:100E4000F602B767004083A707C5B73600208906BA
:100E5000C207C183B697860723A007009307000344
:100E6000239AF18623200700114983A74186238412
:100E700027016FF08FADC147239AF1861D49F5B761
:100E8000DE28114963F38700094963F387003E8434
:100E90009C4C4204418022858297AA8A0145EF003A
:100EA00050572286AA855685EF003030A28501452D
:100EB000EF00D0599E280D67818F9EA8BE283E94D2
:100EC00093070003239AF186A2A82399E18671BFB4
:100ED00083A7418683C69181B833094563E0E60262
:100EE000B42389EED62399EAEFF28FA4B8A783A79B
:100EF000C186DC43829701456FF0CFA58280EFF277
:100F00002FA383A7418603A781864111AC33184FD5
:100F1000C833029783A74186B8270DC72AC61DE1AB
:100F2000D8230DE3BC2399EF83A7C186DC478297C2
:100F300083A741863245D833B8B7B833D8A7410123
:100F40006FF04FA10945E5BF83A74186942393F62F
:100F5000F60781EA98371377F7FD98B701473A8586
:100F6000828009460947E39CC6FEB623EDFAD423E6
:100F7000FDF6EFF2EF9BD03337670040130707C051
:100F80001375F6F7131425003A946206144061862F
:100F90006356060493F6060383C581810947637C83
:100FA000B50295CABC2785CB1C40635C060293F74B
:100FB00007034147639CE7001374F50F2285EF0098
:100FC000303E930500032285EF00502583A7C1869C
:100FD000DC4B829701473A856FF0CF970D67F98E0A
:100FE00065BFC164FD140D67E58FF98F0567E39F49
:100FF000E7FC1DEDB707002083C58709EF00F04629
:101000001C4071771307F7F8F98FC2070D67C1838A
:10101000B98F617713070708D98FC207C1831CC036
:101020008D661840658F758FE302D7FA1CC0D5BF57
:10103000EF00D0331C4071771307F7F8F98FC20720
:101040000D67C183B98F617713070708D98FC2076E
:10105000C1831CC08D661840658F758FE308D7F675
:101060001CC0D5BF03A64186B7670040938707C061
:10107000543293F5F6F713972500BA97E206984392
:10108000E18663DF06041377070303C881810945FE
:1010900063F705092E22C1E559C3382649C3EFF28B
:1010A0002F89984363D30604E5769386F6FB758F04
:1010B00042074183E1761347070193860608558F5F
:1010C0004207418398C34146944393F60603639CC9
:1010D000C60083A7C1869C4F829701456FF08F871A
:1010E0000D65698F5DB798C3C5B7F1769386F6F83D
:1010F000758F420785664183358FE17693860608B2
:10110000558F42074183416698C37D160D658565FD
:101110009443F18EE98EE38EB6FA98C3D5BF8280F0
:10112000EFF20F8103A741861C3793E707021CB734
:1011300083A7C186DC4F829701456FF0AF8103A77B
:1011400041863E2B11E5CA211D8D0AAB01458280E7
:1011500088413E958280EFE2BFFDB707002083C53E
:1011600087090145EF00703083A741868827A14792
:101170006318F50005672399E1864147239AE186C4
:101180005D15133515006FE0FFFCEFE27FFA03A950
:10119000418637660040832706C583468900254778
:1011A00041116385E60441641307F4FFB73600205C
:1011B000F98F9106B69786078043798C060432949E
:1011C0001C202300F9001C30A300F9004A20EF0086
:1011D00010342311A9000A2403A94186EF003033FB
:1011E0002312A9005A2483A74186FAA383A7418624
:1011F000054798A7FA238033631A070C98231377BF
:10120000F7075DE325476315E400D9312DE135A0EB
:1012100015476317E40403873700635A0700A147A3
:1012200003A741861CA7053F41016FE0BFF2B82329
:101230007DF7DA236DF7BC27FDF3B767004083A77E
:1012400007C5373700200907C207C183BA97860749
:1012500023A0070013070003239AE1869947C9B723
:101260000D476315E402B4330547638DE60083A799
:1012700081862285DC4B82970D47A547E302E5FA7C
:101280004DDD71BFDE23E5F7613D49B70547E3104A
:10129000E4FEB833E31D87FCDA2371FB9C3793F738
:1012A0000702F1D755319DB785476317F700AD4762
:1012B000E31FF4FAA93199BF8946E31AD7FAE30389
:1012C000F4FE8D47E315F4FA713B89B719476319AA
:1012D000E40298231377F70771EBBC23854603A735
:1012E00081866395D7005C4FF1C389A089466394DA
:1012F000D7001C53D5BF8D46639AD70A5C53EDB710
:1013000061E8BA2345E7D843C1769386F60F758F17
:10131000B7060200631CD70898231377F70705EF79
:10132000DE23C9E7B7170000938707D903A74186D3
:101330000145231907001CCF8297014583A74186E9
:10134000C166FD169A2B630FD70689466303D50045
:1013500069EF21478DA88546631ED70003A78186C4
:10136000C8338145184F029731E183A74186BC27D6
:10137000D5FB2DA88946631BD702D833B76600403A
:10138000938606C01376F70093172600B6979C4302
:1013900093168701E18663DA060293F7070383C693
:1013A00081816375D6001377070779D303A7418638
:1013B00083A7818608339C4B82978D47E310F5F80D
:1013C00083A74186254798A7B9BD8D66F58FC1BF14
:1013D0002147631BE4009C2393F7F707E1FBB71752
:1013E00000009387C7D499B72947E311E4FC9823F9
:1013F00085461377F707E31BD7FAB82745DBBA23EF
:1014000055F7D843C1769386F60F758FC166E31FF3
:10141000D7F803A78186C8338145184F029759F53D
:10142000B71700009387E7D611B78386070063D20A
:10143000060483A68186EE2303C6C6022EC6324565
:1014400093160601C1826378E50032479AABD6ABAA
:10145000EFF01F9DC9BBE37CB7FE6375D70023AED9
:101460000184F5B73367C7027DF3054623AEC18417
:10147000F9BF0D4798A70D672399E1866DB3EFE299
:101480009FC903A44186A1441C241387E7FF137757
:10149000D70F25C71387D7FF1377D70F49EF1C4CFA
:1014A00085CB0628B1C05A2863739700BA84C2045A
:1014B000C180268582971E28AA890145858F1EA88E
:1014C0003E28A6973EA8A527AA8526864E850123F5
:1014D0001E2899CB0D67814501452399E186BD27DB
:1014E00013070003239AE1861E28562803A7418686
:1014F00063ECD7008D471CA7042783A7418684A7E8
:10150000EFF07FC56FE07FC499C39547EDB799476A
:101510001CA7B767004083A707C5B7360020890618
:10152000C207C183B697860723A00700930600036E
:10153000239AD186D1B71D47A144E390E7FC83A746
:101540008186DC47829755BF03C38181376600409F
:10155000C1650568A1680147130606C0FD1513089B
:10156000F8F0938808086369670013650508B76792
:10157000004023A6A7C4828093162700B2969C42FF
:10158000ED8FB3F70701D98FB3E717019CC20507A9
:10159000D9BFEFE2FFB983A7418694271387E6FFFF
:1015A0001377D70F09EFEFF0BF8783A741869827FE
:1015B00083A7418698A7EFF01FBA6FE0BFB919461D
:1015C0002147E397C6FE94331547639CE6009823B2
:1015D0001377F70719E7A833853F83A7C1869C5384
:1015E000829783A781869C4782972147D1B78280C3
:1015F000EFE29FB14111370A0020B70A0020E179DC
:1016000023170100130A4A03938A0A0593890908DC
:10161000B765004083A745C413970701418323940E
:10162000E188139707016357071683D781883A84A7
:10163000BD8B2381F186938605C06397073003A78E
:1016400005C093872187420741839AA39A239386F3
:101650004187137707039AA29A238D662166758FB7
:101660009AA303A705C0A5679387F7FB7D8F83A780
:1016700005C0B1669386F6F8F58F8966B58F134776
:10168000070293160701130606085D8F518FC1826A
:1016900023A0E5C033E736014207938421871389ED
:1016A000418737660040930500024183832606C0C8
:1016B00093F606036393B60EB3E73701C166C2071C
:1016C00037660040FD160D658965C183032706C096
:1016D000130406C0758F698F6314B70C83D7818894
:1016E000C18BE1EB1C40A5691387F9F0F98F1CC091
:1016F0004D3518401440B1679387F7F8F58F962061
:101700009389F9FB3377370113963601635406004A
:101710008566B58F96201396260163540600896668
:10172000B58F83560900C18A99C2134707018356B2
:10173000090093F6060299C2134707022166931621
:101740000701130606085D8F518F3766004023207E
:10175000E6C06177C18213070708558F42074183AE
:10176000832606C08355090093F60603639DB602DF
:10177000617713070708D98FC166C2073766004033
:10178000FD160D65C183032706C08E20758F698FF6
:10179000631EB70041016FE0BF9A2320E6C039B74E
:1017A0002320F6C025B72320E6C05DBF2320F6C066
:1017B000D9BF1C40856BC207C1837C873C871397C8
:1017C00047016350070C1C401387FBF8F98F1CC0BE
:1017D000EFF0BF9B1840A5679387F7FB14407D8F00
:1017E000B1679387F7F8F58F962013963601635407
:1017F0000600B3C7770196201396260163540600AE
:101800008966B58F83560900C18A99C213470701BB
:101810008356090093F6060299C213470702216610
:1018200093160701130606085D8F518F3766004037
:101830002320E6C06177C18213070708558F42074E
:101840004183832606C08355090093F606036397F8
:10185000B602617713070708D98FC166C2073766DA
:101860000040FD160D65C183032706C08E20758FCD
:10187000698FE301B7F22320F6C0FDB72320E6C04D
:10188000C9B73C87C207C187E3D407D81C40138778
:10189000FBF8F98F1CC0EFF09FBE1840A567938737
:1018A000F7FB14407D8FB1679387F7F8F58F96208B
:1018B0001396360163540600B3C77701962013963A
:1018C0002601635406008966B58F83560900C18AD4
:1018D00099C2134707018356090093F6060299C27D
:1018E00013470702216693160701130606085D8F4A
:1018F000518F376600402320E6C06177C18213070D
:101900000708558F42074183832606C08355090087
:1019100093F606036397B602617713070708D98F1A
:10192000C166C20737660040FD160D65C1830327F7
:1019300006C08E20758F698FE30EB7E42320F6C0B2
:10194000FDB72320E6C0C9B7139727003697144385
:10195000C206C18274873487C206C18663DD060071
:10196000FD1714438A070566D6971306F6F89C43BD
:10197000F18E14C382973C8793F70708E38A07C860
:1019800083C72186B7660040938606C01397270059
:101990003697FD1714438A07D29725661306F6F08B
:1019A0009C43F18E14C38297A5B1B737002005067A
:1019B000BE950586860511E282801C3118219105AD
:1019C000A207D98F239EF5FE09057D16EDB7B7371F
:1019D00000200506BE950586860511E282809C41A1
:1019E00009057D16231FF5FE9105C5BF61994205C6
:1019F0004181B767004023A8A7C48280B767004031
:101A0000938707C00A053E951C4165771307F79831
:101A1000F98FDD8DC205C1810CC18280B76700409E
:101A2000938707C00A053E951C4165771307F7FBAE
:101A3000F98FC20713F70501C18319C393C70701C3
:101A400013F7050219C393C7070261771307070845
:101A5000D98FC207C1831CC1184113770703E31C48
:101A6000B7FE8280B7670040938707C00A053E959E
:101A70001C4171771307F7F8F98FC20713973501E7
:101A8000C183635407000567B98F13972501635419
:101A900007000967B98F617713070708D98FC20755
:101AA000C183C1661CC1FD160D661841758F718F0B
:101AB0006313B70082801CC1CDBFB7670040938716
:101AC00007C00A053E951C4165771307F7FBF98FA0
:101AD000C207C183617793C7070313070708D98F2C
:101AE000C207C1831CC19306000318411377070383
:101AF0006313D70082801CC1CDBFB76700409387B6
:101B000007C00A053E951C4171771307F7F8F98F56
:101B1000C2070D67C183B98F617713070708D98F93
:101B2000C207C183C1661CC1FD160D661841758FC1
:101B3000718F6313C70082801CC1CDBFB76700409F
:101B4000938707C00A053E951C4105671307F7E018
:101B5000F98F617713070708D98FC207C1831CC1AA
:101B60008280EFE2EFDCD93F6FE0CFDEB767004065
:101B7000938707C00A053E951441C1671387F7FF95
:101B80009397160163DD07001C41F98F0567130762
:101B9000F7F0F98F316713070708D98F1CC18280CE
:101BA000B7670040938707C00A053E951C4193F72D
:101BB000070491CF1C4141677D17F98F0567130713
:101BC000F7F0F98F21671307070CD98F1CC18280AA
:101BD000B767004083A707C50E058581C207C1838B
:101BE0003E95B73700203E95060586050CC18280DC
:101BF000B767004083A707C50E058581C207C1836B
:101C00003E95B737002091073E95060586050CC125
:101C10008280B767004083A707C50E05C207C1834E
:101C20003E95B73700203E9506050A218280B767AA
:101C3000004083A707C50E05C207C1833E95B7378D
:101C4000002091073E9506050A218280B767004073
:101C500083A707C50E05C207C1833E95B73700208D
:101C600089073E9506050CC18280B767004083A7AF
:101C700007C513173500C207C183BA97373700204D
:101C80001907BA971307E00386076373B70413D7DE
:101C90005500FD8981E57D17420741832A07A1662A
:101CA000558F98C30DE5B707002083C78709130731
:101CB000E0036376F70213D75700FD8B81E77D17AA
:101CC000420741832A07E1775D8F239DE186828069
:101CD00013D71500858991C105072A07D9B713D7EE
:101CE0001700858B91C305072A07C5B7B767004062
:101CF00083A707C50E05C207C1833E95B7370020ED
:101D000099073E95060508411375F53F8280935764
:101D100085001375F50F22055D8D828037670040C1
:101D2000F177232207C4938707F02398F186B167E0
:101D3000938707F02320F7C401458280EFE24FBF6D
:101D400032849374F507268542042E894180D1356B
:101D50002286AA854A85EFF05FC52685A285FD35D6
:101D600001456FE02FBFEFE2AFBC9374F507268506
:101D70002E89AD3F2A8426855D3DAA8522864A8527
:101D8000EFF0FFC422856FE0EFBC37050400EF00E1
:101D9000104D73002030E12A730020300D4723AA34
:101DA000E188828003C761D609C7154723AAE18865
:101DB00082800547E5BFEFE2AFB7AA842E841145C4
:101DC0008545EF00B072B1CCB766004083A706C46A
:101DD00041677517F98F23A0F6C4B717014003A711
:101DE0004780B716F0FFFD16758F23A2E78003A783
:101DF000C780F9769386F67F758F23A6E78003A7C1
:101E00004780B7460400558F23A2E780374702403A
:101E10008327078021C893E727002320F7806FE0FE
:101E20006FB337670040832707C4B716F0FFFD166E
:101E300093E72700C207C1832320F7C4B7170140E7
:101E400003A74780758F23A2E78003A7C780F97691
:101E50009386F67F758F23A6E78003A74780B73662
:101E6000030055B7F59B55BF8280EFE2CFAA3971C9
:101E70000945AD3D2A8A09455D3BAA8552860A85FA
:101E8000EFF0FFB41387418A74237C3313070040BB
:101E9000B70A0020A207D58FB307F7401384418A01
:101EA000938ACA1A0A896344FA047C20643093092D
:101EB0000040CA85A204DD8C7C206830B38999403B
:101EC000C20922055D8D93D909014E8656959384EA
:101ED00004C0EF10E01ED2947C20139A0401230367
:101EE00004007C304E99A3030400135A0A017C209D
:101EF00068305286CA8522055D8D5695EF10401CCC
:101F00000945EFF09FBF21616FE02FA4238B01866D
:101F10009387418A238C070282808280EFE24FA15F
:101F2000938581D7130540083D3D13160501418275
:101F3000239CC186138781D781476311F60213164C
:101F400005014182938581D71145CD3B1145EFF0C5
:101F5000DFB61145EFF07FBA6FE0CF9F14238507FE
:101F6000C20793C6F6FF14A3C1830507F9B7EFE2D2
:101F70002F9C37680040032708C5C1651385F5FF0E
:101F800083D6A187B7370020698F13866700329701
:101F900006071843938505C00111F98D638CD500A0
:101FA000832708C593F606C0E98FB2978607984342
:101FB000D98E94C3B766004083A746C4138781882F
:101FC000C207C1831EA31A2383D701871384818884
:101FD0007D8F1377072009CF41671307F7DF23A20F
:101FE000E6C49386C187982205071377F70F98A256
:101FF0001A20F98FC207C18763D40700EFF04FDFC3
:102000001E2003D70187F98F93F7074089CFC16757
:102010009387F7BF376700402322F7C4B707002034
:1020200083A7070782971A2083D701877D8F93168E
:10203000270163D806003967B76600407D1723A2E1
:10204000E6C41A20F98F13973701635B0700BD6759
:1020500037670040FD172322F7C40145EF00806F6A
:1020600003D701871E20F98F13974701635007029A
:1020700083C7C18293F7F70F638F070ECD2BBD6720
:10208000376700409387F77F2322F7C41E2003D7CA
:102090000187F98F93F70710E1CFC16737670040D9
:1020A0009386F7EF2322D7C4032687C4938601883B
:1020B0009315060163DA050A9042050690C28C4228
:1020C0000D466375B60A032607C4FD17218A59EE2B
:1020D000032607C4938541887D8E3765004090C1F3
:1020E000138741880146130305C0A14893152600B4
:1020F00033886500032808000010A2953378F800A3
:1021000023A005FF0506E31316FF10431366160010
:1021100010C310437D8E2320C5C41043799A10C389
:102120001843F98F2320F5C437670040832747C43D
:1021300093F70740E5DFC1679387F7BF3765004036
:10214000C1652322F7C4130505C08147FD15214849
:102150001397270010103A96032606FE2A97850744
:102160006D8E10C3E39607FF23A006001D45DD23F7
:1021700005616FD03FFE0945F12B11B791E5854709
:1021800033B5A700060582800945828011E583A743
:1021900041861D479AAB82801385018E8280EFD2E3
:1021A0003FF9ED376FD01FFBEFD29FF883A6418632
:1021B0000546BA849C2293F7F7076392C704BC22B2
:1021C000130720026388E702130710020945639191
:1021D000E702372400001304245C80CE01450294FA
:1021E00083A74186014580CF2399070002940145CA
:1021F0006FD05FF6372400001304245BF9BF130788
:1022000010020945E396E7FE9832630BF700930747
:102210000002E31FF7FC372400001304E419C9B7D8
:10222000372400001304C41865BF03A74186930632
:10223000100201451C3318231377F707631AD700E0
:102240009387E7FD93F7F70F05453335F50006054E
:10225000828003A74186930610021C2393F7F70799
:10226000639DD7001833930700026318F700EFD27D
:102270003FECEFD07FF96FD0FFED8280EFD25FEBC4
:102280000D670347771883A74186014598B72395C3
:102290000700EFF0AFF5930500200145EFF00FF6D2
:1022A000C1450145EFF08FF7930500040145EFF0BC
:1022B0003F94930500080145EFF09F910145EFF031
:1022C0005F8AB707002083C587090145EFF0FF99B2
:1022D0000145EFF09F8237670040032607C0C167C2
:1022E0009386F7FF9317160163DF0700832707C064
:1022F000F58F85669386F6F0F58FB16693860608AE
:10230000D58F2320F7C037670040832707C093F796
:10231000070485C3832707C0C166FD16F58F856650
:102320009386F6F0F58FA1669386060CD58F232051
:10233000F7C0930500600545EFF04FEC93050002F0
:102340000545EFF0AFED9305000C0545EFF05F8814
:1023500081450545EFF00FF137670040832747C0FF
:1023600093F7070485C3832747C0C166FD16F58F21
:1023700085669386F6F0F58FA1669386060CD58F59
:102380002322F7C037670040032647C0C167938602
:10239000F7FF9317160163DF0700832747C0F58F08
:1023A00085669386F6F0F58FB16693860608D58F1D
:1023B0002322F7C081450945EFF04FE481450945E7
:1023C000EFF0CFE5930500100945EFF07F8293050C
:1023D00000040945EFF07F898D650945EFF08FE82E
:1023E00037670040032687C0C1679386F7FF9317BE
:1023F000160163DF0700832787C0F58F8566938604
:10240000F6F0F58FB16693860608D58F2324F7C0C2
:1024100037670040832787C093F7070485C3832766
:1024200087C0C166FD16F58F85669386F6F0F58F39
:10243000A1669386060CD58F2324F7C081450D45F0
:10244000EFF0CFDB930500020D45EFF02FDD930594
:1024500000140D45EFF0CFF781450D45EFF08FE00B
:10246000376700408327C7C093F7070485C38327D6
:10247000C7C0C166FD16F58F85669386F6F0F58FA9
:10248000A1669386060CD58F2326F7C037670040D8
:102490000326C7C0C1679386F7FF9317160163DF52
:1024A00007008327C7C0F58F85669386F6F0F58F02
:1024B000B16693860608D58F2326F7C09305006082
:1024C0001145238B0186EFF06FD393050002114570
:1024D000EFF0CFD4930500181145EFF06FEF93059F
:1024E000001C1145EFF0CFF0930500041145EFF00B
:1024F000CFF78D651145EFF0EFD6376700408327A2
:1025000007C193F7070485C3832707C1C166FD167A
:10251000F58F85669386F6F0F58FA1669386060C97
:10252000D58F2328F7C037670040032607C1C1674E
:102530009386F7FF9317160163DF0700832707C110
:10254000F58F85669386F6F0F58FB166938606085B
:10255000D58F2328F7C00145EFE01FFF0547238BE8
:10256000018623AAE1886FD0FFBEEFD27FBC93859E
:102570000181EFE0DFBC6FD0FFBDEFD27FBB938561
:102580008180EFE0DFBB6FD0FFBC83A74186AC3317
:10259000914763EEB700EFD2BFB9B707002093872A
:1025A000C7098E05BE95EFE09FB96FD0BFBA014550
:1025B0008280EFD2FFB793854182EFE05FB86FD0A2
:1025C0007FB9EFD2FFB69385C181EFE05FB76FD0DF
:1025D0007FB8EFD2FFB583A741864111238507005D
:1025E0009520B7670040856637660040938707C02F
:1025F0009386F6F0930506C298439107758F23AE34
:10260000E7FEE39BB7FE9307F00F2322F6C4EFF03B
:10261000EFF08145014523AA0188EFF0CFF9B70714
:10262000002083A7470C95833EC6B24781EB8545C2
:102630000545EFF04FF841016FD0DFB1B247FD170C
:10264000E5B78280B7670040054723A0E7C423A011
:1026500007C4096723A207C4130707C02398E186AC
:102660000967130707C023A0E7C401458280EFD2A2
:102670003FACB767004083A707C437670040416895
:10268000C207C1838146130307C07D18938581DB90
:10269000A148139626003305660008412E9685064C
:1026A0003375050108C2E39616FF93E60740232021
:1026B000D7C493E61740F99BC207C1832320D7C430
:1026C00093E607402320D7C4B766004003A746C45B
:1026D0001377074065DF41671307F7BF23A2E6C4FE
:1026E0004168376700408146130307C07D18A14841
:1026F000139626003385C50008411A968506337562
:10270000050108C2E39616FF93E787402320F7C42C
:10271000832707C4C207C18393E747002320F7C478
:10272000EFF0CFE76FD01FA3EFD29FA03764004038
:10273000832704C4C207C183ED9BC207C183232042
:10274000F4C4EFF02FE6B167938707F02320F4C4B9
:102750006FD05FA0EFD2DF9D9D471384C1886303D4
:10276000F50008C01C401547636DF7000D678A0728
:102770001307C724BA979C43828783A7818981E77F
:102780006537994711A095471CC039A0713F914703
:102790001CC0054723ACE1886FD0DF9B89475CA054
:1027A0008D47DDB75C20FD1793F7F70F5CA05C2029
:1027B00093F7F70FF5F39147C1BF376700408327C1
:1027C00007C4C207C18393E707012320F7C49547D5
:1027D0001CC0A9475CA0C9B75C20FD1793F7F70F91
:1027E0005CA05C2093F7F70FC5FB37670040832799
:1027F00007C4C207C183BD9BC207C1832320F7C49E
:1028000099471CC023AC018841BF01A097E1FF1F7D
:102810009381410B172100201301C17E1715000081
:10282000130585A497D5FF1F9385C57D1386018465
:1028300063FAC5008322050023A055001105910508
:10284000E3EAC5FE13850184938581DD6377B500D6
:10285000232005001105E36DB5FE73D00FBC73D0C6
:102860004180930280087390023097D2FFFF9382D9
:10287000A27993E2320073905230EFE0CFB997E241
:10288000FFFF938282177390123473002030EFD2CF
:102890003F8AB727014093870740631CF5008545B1
:1028A000130500205121814513050020B5296FD063
:1028B0007F8AB737014093870780E31AF5FE854585
:1028C000130500409521814513050040C5B75C41C3
:1028D0003707F1E01307F7EF944D7D8F9C41D58FBB
:1028E000D44DD58FD441A206D58FD98F5CC11C455C
:1028F00037F7F1FF1307D77FD4457D8F9C49D58FDC
:1029000094458606D58FD98F1CC55C55370710FFB7
:102910007D177D8FDC29FD1793F7F70FD207D98F2D
:102920005CD582801C4589C593E717001CC5828051
:10293000F99BEDBF1C4591C537075000D98F1CC5C9
:1029400082803707B0FF7D17F98FD5BFA54763F7A2
:10295000B7048D47138765FF3307F7020328C500C7
:102960009D47B397E70093C7F7FFB3F70701B39607
:10297000E600DD8E54C5994763E3C70495477D168D
:102980003306F6025859FD47B397C70093C7F7FFC0
:10299000F98F3396C5005D8E50D982800D473387FD
:1029A000E502032805019D47B397E70093C7F7FFAA
:1029B000B3F70701B396E600DD8E14C96DBFB147CA
:1029C00063E2C702954765163306F6021859FD47BC
:1029D000B397C70093C7F7FFF98F3396C5005D8E95
:1029E00010D9828095474D163306F6025855FD479B
:1029F000B397C70093C7F7FFF98FB395C500DD8D77
:102A00004CD58280684542054181828008416D8DA8
:102A10003335A0008280EFD2AFF105452D26014568
:102A20001D266FD02FF34111B777004002C6938760
:102A300007C03EC6B2473E952AC6B2478CC3410185
:102A400082804111B777004002C6938707C03EC617
:102A5000B2473E952AC6B2478A2341018280B70712
:102A6000014023AAA74082809C4513F7070113F871
:102A7000F70001C7D8413368E80037270240145BEC
:102A80003707000F758F4DEB8546238ED18837179A
:102A900001406315E5009A2135839AA18E2113F731
:102AA000F50F39C318418146854E3D4F930F800283
:102AB00093028004214E3396DE00B3F8C500631103
:102AC00016039398260033131F011343F3FF337744
:102AD000E300B318180133E7E8006397F70750C91C
:102AE0008506E39AC6FD18C11307F00F6375B70496
:102AF00054412146854E3D4F930F8002930280043E
:102B0000414EB398CE0033F715016392E8021317D4
:102B1000260001173313EF001343F3FFB376D300FE
:102B20003317E800D98E6395F703232A15010506AC
:102B3000E319C6FD54C1828037170140E310E5F662
:102B400003C7C18921DF81BFE39C57F810C949BF82
:102B5000E39F57FC23281501D9BFB7070140635AEB
:102B60000504DC4F935605011318050137073000A3
:102B700013F6F60013580801B376E500635E050608
:102B80006399E604930606010D46B316D60093C674
:102B9000F6FFF58F99C9135755011377F73F1207C1
:102BA0003317E800D98F63550506370701405CCF1E
:102BB000828037270240145BDC433707000F758F94
:102BC00055F313D71700F976CE07758FCD83D98FBC
:102BD00051BF1317B500635607008D46B396C60064
:102BE0007DB7135755011377F73F12073317E800E6
:102BF0001347F7FFF98F79BF6390E602370601406C
:102C00005442370700F17D17F98F758F58C2C1F50F
:102C1000370701405CC382801317B500635C07006F
:102C20008D46B396C60093C6F6FFFD8EB707000F1C
:102C3000D58FF1BF1357550112073317E80013471B
:102C4000F7FF7D8FB707000FD98FD1B723A0A18AD7
:102C50008280377700401C4309C593E707101CC3E7
:102C6000828093F7F7EFE5BFB7160240DC42517759
:102C70007D17F98F5D8DC8C28280B717024023800F
:102C800007022380070205476306E5001147630634
:102C9000E50082802380A702828015472380E70217
:102CA0008280371702401C535D8D08D3828001C992
:102CB000371702401C53A166D58F1CD38280B716EC
:102CC00002409C5261777D17F98F9CD2828099C512
:102CD000371702405C4B5D8D48CB8280B7170240AE
:102CE000D84B1345F5FF798DC8CB828099C537172E
:102CF00002401C4F5D8D08CF8280B7170240984F6D
:102D00001345F5FF798D88CF828099C5371702402A
:102D10005C4F5D8D48CF8280B7170240D84F134576
:102D2000F5FF798DC8CF828099C5371702405C477F
:102D30005D8D48C78280B7170240D8471345F5FF1D
:102D4000798DC8C7828001C9371702401C53C166FC
:102D5000D58F1CD38280B71602409C5241777D17D5
:102D6000F98F9CD282809357550005476399E700FD
:102D7000B71702409C4333D5A700058982800947D5
:102D80006396E700B71702409C53F5B7B7170240A8
:102D9000DC53D5B7B737004003D747801367070127
:102DA0002392E78082803737004083574780C207ED
:102DB000C183BD9BC207C1832312F7808280EFD2FB
:102DC0002FB741112AC6F9373245B737004013579C
:102DD00005014205239CE7804181239EA780E137BE
:102DE00041016FD02FB7EFD2AFB441112AC6EFF037
:102DF0007FFA3245B7370040135705013D8B420536
:102E00002394E78041812396A780EFF0DFF9410109
:102E10006FD04FB4373700408357478093F707028E
:102E2000E5DF82803737004083574780C207C18380
:102E3000DD9BC207C1832312F780373700408357D9
:102E40004780A18BEDDF82801E21373701401307B9
:102E500007C0C207C1836304E5023707004063006F
:102E6000E50213070740630CE5003717004093069F
:102E700007806306D500130707C06316E500BA2173
:102E800093F7F7F8D98FFA2193F7F7CFC207C183E9
:102E9000D98F1EA1DE215EB59E211EB5B737014038
:102EA000938707C06314F5009C251EB985475EA96A
:102EB00082801E31922103D82500C207C183F99B6D
:102EC000C207C1831EB11E3156211A2DC207C1830C
:102ED000420741831377C7F8518F9225F59BC206AD
:102EE00033660601D18F37360140130606C0C18212
:102EF0006310C502B225DD9B03D8E500D18FD22136
:102F0000ED9B93F6F6CFD18FD22533660601D18E95
:102F100056A11AADFA215AB91EB182801E316577C9
:102F20001307F7CFC207C183BD9BC207C1831EB180
:102F30001E31562103D88500C20713960601162DAF
:102F4000C18393F7F7FD758F96214182A206558FB5
:102F5000B62142074183B3E606019206D58FB73604
:102F60000140C207938606C0C183631ED502B62501
:102F700093F7F7F703D8C5009206D58FD621C2077D
:102F8000C183920693F7F7FBD58FFD769386F63FC4
:102F9000F18EF225C207C183336606010A06D18E7F
:102FA00013960601418252A11AADFA211ABD1EB133
:102FB00082801E3103D88500C207C18393F7F7EFE3
:102FC000C207C1831EB11E3156215A2DC207139666
:102FD00006014207962141831377C7F8558FB62122
:102FE000C18393F7F7DFB3E60601A206D58FB736A4
:102FF0000140C207938606C04182C183631FD50288
:10300000FD769386F67FF58FB62503D8C500A20618
:10301000D58FD621C207C183A20693F7F7BFD58FFC
:10302000F576FD16F18EF225C207C18333660601DF
:103030001206D18E13960601418252A15AADFA2191
:103040005ABD1EB182801E2189C593E717001EA1BB
:103050008280C207C183F99BC207C183CDBF83575A
:10306000450491C52167D98F2312F5048280C607D4
:10307000C583DDBF1E2189C593E707081EA1828095
:10308000C207C18393F7F7F7C207C183C5BF1E2DDF
:10309000C207C183DD9BDD8D0EAD82801A2DFD77C9
:1030A0009387F77FF98FA205CD8FC207C1831EAD2D
:1030B00082805E2DC207C183DD9BDD8D4EAD828097
:1030C000B3C7A5008D8B3307C50081E78D4763ED3E
:1030D000C700AA87637EE508942185078505A38F2D
:1030E000D7FEE3EBE7FE828093763500AA8789CA94
:1030F000942185078505A38FD7FE93F63700C5BFBA
:103100009376C7FF138606FE63F0C70683A3050008
:1031100083A2450083AF850003AFC50083AE0501E0
:1031200003AE450103A3850183A8C501938545022C
:1031300023A0770003A8C5FF23A2570023A4F7010B
:1031400023A6E70123A8D70123AAC70123AC670060
:1031500023AE17019387470223AE07FF75B790414F
:103160009107910523AEC7FEE3EBD7FEE3E6E7F652
:10317000828000001F1C1F1E1F1E1F1F1E1F1E1FE0
:1031800009026B000301008032080B0002020201F9
:1031900000090400000102020100052400100105DD
:1031A0002401000104240202052406000107058110
:1031B0000340000109040100020A000000070502A3
:1031C00002400000070583024000000904020002DB
:1031D00003000000092111010001222200070584DB
:1031E0000340000107050403400001001201100123
:1031F00000000040861A0CFE0001010200010000E0
:103200000600FF0901A101090226FF00750815004B
:10321000954081060902150026FF0075089540912A
:1032200006C0000016035500530042002000530062
:1032300065007200690061006C0000000E037700F9
:10324000630068002E0063006E0000007A27000013
:103250008C2700009C270000A4270000BA2700004C
:04326000D82700006B
:103264002000000002000000100000000000000028
:1032740000000000010203040607080916033000D9
:103284003100320033003400350036003700380096
:1032940039000000681E0000EE1500000C1F00003D
:1032A4001A1F0000EE150000EE150000EE150000D8
:1032B400EE1500006A1E0000EE1500001C1F000041
:1032C400EE150000EE150000EE150000D2250000FA
:1032D4007C2200005222000042260000A8210000A7
:1032E4002A2200007C2100006A2500007A250000C3
:1032F4008A2500000000000040000000F8000020C3
:10330400040000003C3200000E00000024320000E3
:10331400160000001C000020160000000000000041
:1033240001000000006CDC02803100006B00000032
:10333400EC310000120000000F010000D431000045
:10334400090000000032000022000000010000001B
:10335400E8070B0108000000040309040000000052
:00000001FF
